:04000000F9EF00F024
:10000800FFFFFACF20F0FBCF21F0E9CF22F0EACFB3
:1000180023F0E1CF24F0E2CF25F0D9CF26F0DACFD4
:1000280027F0F3CF28F0F4CF29F0F6CF2AF0F7CF56
:100038002BF0F8CF2CF0F5CF2DF0F2A201D001D0A3
:10004800AAD0F292F29A92D0010E606E9AD0860EE1
:10005800595C000E5A58D8A001D001D00AD08A0E97
:10006800595C000E5A58D8B001D001D002D0020E07
:10007800606E000E5D6E000E5F6E83D0090E595CD7
:10008800000E5A58D8A001D001D06BD0190E595C77
:10009800000E5A58D8B001D001D063D0090E595C6F
:1000A800000E5A58D8A001D001D00AD00D0E595CC4
:1000B800000E5A58D8B001D001D002D019D018D0AB
:1000C800130E595C000E5A58D8A001D001D00CD09C
:1000D800190E595C000E5A58D8B001D001D004D07E
:1000E8005F5080095F6E04D0010E606E4AD000D068
:1000F8005D2A5D50070BD8A401D001D02ED05DC079
:1001080008F0096A000E0B6E080E0A6E08EC05F07E
:10011800FF0E0826530E0824D96EDA6A000EDA227A
:100128005FC0DFFF000E5F6E1F0E5D6401D001D05F
:1001380014D0000E606E000E5D6E010E5E6E55C02E
:1001480051F053C01AF054C01BF055C01CF056C0F3
:100158001DF065EC07F001D000D0D8905F305F6EDD
:1001680010D0000E606E0DD00CD00BD06050000A7D
:10017800D8B46AD7010AD8B46AD7030AD8B47ED7E4
:1001880000D0F28A000ED76E9C0ED66E000E5A6E04
:10019800000E596E00D0F2A401D001D008D0F2941C
:1001A800594A5A2A9C0ED626000ED72200D02DC0B6
:1001B800F5FF2CC0F8FF2BC0F7FF2AC0F6FF29C0B7
:1001C800F4FF28C0F3FF27C0DAFF26C0D9FF25C0F7
:1001D800E2FF24C0E1FF23C0EAFF22C0E9FF21C0FB
:0E01E800FBFF20C0FAFF1100FFFFFAEF07F047
:100600003031323334353637383941424344454648
:10061000495220526563697665642054657374009D
:100620005F000000FFFF000E196E000E186E030E33
:10063000046EE80E036E11C001F012C002F0BEECB1
:1006400005F001C008F002C009F0000E0B6E640E48
:100650000A6E08EC05F008C014F009C015F0000E91
:10066000046E640E036E11C001F012C002F0BEEC05
:1006700005F001C008F002C009F0000E0B6E0A0E72
:100680000A6E08EC05F008C016F009C017F011C09A
:1006900001F012C002F0000E046E0A0E036EBEECF2
:1006A00005F001C018F002C019F0630E1424D96ED1
:1006B000DA6A000EDA22DF50036EE4EC03F0630E18
:1006C0001624D96EDA6A000EDA22DF50036EE4ECEB
:1006D00003F0136E2E0E036E1350E4EC03F0630E62
:1006E0001824D96EDA6A000EDA22DF50036EE4ECC9
:1006F00003F01200FFFFFFFF000E466E000E456E76
:10070000030E316EE80E306E3EC02EF03FC02FF06B
:1007100068EC05F02EC035F02FC036F0000E386EB4
:10072000640E376EA8EC04F035C041F036C042F0DC
:10073000000E316E640E306E3EC02EF03FC02FF0C2
:1007400068EC05F02EC035F02FC036F0000E386E84
:100750000A0E376EA8EC04F035C043F036C044F002
:100760003EC02EF03FC02FF0000E316E0A0E306EEC
:1007700068EC05F02EC045F02FC046F0630E412412
:10078000D96EDA6A000EDA22DF50306E46EC04F0E1
:10079000630E4324D96EDA6A000EDA22DF50306E1F
:1007A00046EC04F0406E2E0E306E405046EC04F0E5
:1007B000630E4524D96EDA6A000EDA22DF50306EFD
:1007C00046EC04F01200FFFFFFFF0350F00B01099D
:1007D000626E046E030E016E045062C002F02FECD4
:1007E00008F06284046E030E016E045062C002F0D1
:1007F0002FEC08F06294046E030E016E045062C088
:1008000002F02FEC08F0040E046EE50EE82EFED781
:10081000042EFCD700F06290046E030E016E0450AB
:1008200062C002F02FEC08F00338F00BF00B010966
:10083000626E046E030E016E045062C002F02FEC73
:1008400008F06284046E030E016E045062C002F070
:100850002FEC08F06294046E030E016E045062C027
:1008600002F02FEC08F0040E046EE50EE82EFED721
:10087000042EFCD700F06290046E030E016E04504B
:1008800062C002F02FEC08F01200FFFFFFFF3050B3
:10089000F00B0109626E316E030E2E6E315062C094
:1008A0002FF025EC08F06284316E030E2E6E31506D
:1008B00062C02FF025EC08F06294316E030E2E6EAC
:1008C000315062C02FF025EC08F0040E316EE50EB9
:1008D000E82EFED7312EFCD700F06290316E030E69
:1008E0002E6E315062C02FF025EC08F03038F00B3E
:1008F000F00B0109626E316E030E2E6E315062C034
:100900002FF025EC08F06284316E030E2E6E31500C
:1009100062C02FF025EC08F06294316E030E2E6E4B
:10092000315062C02FF025EC08F0040E316EE50E58
:10093000E82EFED7312EFCD700F06290316E030E08
:100940002E6E315062C02FF025EC08F01200FFFF30
:10095000FFFF396E000E3B6E395038AE01D001D02A
:1009600009D0376C381ED8B0382A396E010E3B6E6C
:10097000395000D036AE01D001D007D0356C361ECC
:10098000D8B0362A010E3B1A00D0000E3D6E000E84
:100990003C6E38503710D8B401D001D028D0396E11
:1009A000010E3A6E395005D0D890373638363A2A8B
:1009B00000D038AE01D001D0F7D701D000D0D89008
:1009C0003C363D363750355C38503658D8A001D0CB
:1009D00001D006D03750355E3850365A3C8000D0B2
:1009E000D890383237323A2EEAD701D000D03B5077
:1009F000D8B401D001D005D03C6C3D1ED8B03D2A02
:100A000000D03CC035F03DC036F000D01200FFFFF2
:100A1000FFFF0C6E000E0E6E0C500BAE01D001D01D
:100A200009D00A6C0B1ED8B00B2A0C6E010E0E6E8C
:100A30000C5000D009AE01D001D007D0086C091EBF
:100A4000D8B0092A010E0E1A00D0000E106E000E4A
:100A50000F6E0B500A10D8B401D001D028D00C6E04
:100A6000010E0D6E0C5005D0D8900A360B360D2AAB
:100A700000D00BAE01D001D0F7D701D000D0D89074
:100A80000F3610360A50085C0B500958D8A001D018
:100A900001D006D00A50085E0B50095A0F8000D0D2
:100AA000D8900B320A320D2EEAD701D000D00E506A
:100AB000D8B401D001D005D00F6C101ED8B0102AC8
:100AC00000D00FC008F010C009F000D01200FFFFE6
:100AD000FFFF326E000E346E32502FAE01D001D0C7
:100AE00009D02E6C2F1ED8B02F2A326E010E346E14
:100AF000325000D031AE01D001D005D0306C311E63
:100B0000D8B0312A00D031503010D8B401D001D043
:100B100024D0326E010E336E325005D0D89030366C
:100B20003136332A00D031AE01D001D0F7D701D011
:100B300000D030502E5C31502F58D8A001D001D0B9
:100B400005D030502E5E31502F5A00D0D89031321F
:100B50003032332EEED701D000D03450D8B401D08B
:100B600001D005D02E6C2F1ED8B02F2A00D02EC059
:100B70002EF02FC02FF000D01200FFFFFFFF056EF8
:100B8000000E076E055002AE01D001D009D0016CF5
:100B9000021ED8B0022A056E010E076E055000D065
:100BA00004AE01D001D005D0036C041ED8B0042AD5
:100BB00000D004500310D8B401D001D024D0056E69
:100BC000010E066E055005D0D89003360436062A6D
:100BD00000D004AE01D001D0F7D701D000D003502F
:100BE000015C04500258D8A001D001D005D00350B8
:100BF000015E0450025A00D0D89004320332062E0F
:100C0000EED701D000D00750D8B401D001D005D024
:100C1000016C021ED8B0022A00D001C001F002C04F
:100C200002F000D01200FFFFFFFF750E326EF40ECF
:100C3000E82EFED7322EFCD700D000F0326E300EF8
:100C4000306E3250AEEC06F0140E326E7D0EE82E91
:100C5000FED7322EFCD700F0326E300E306E32509E
:100C6000AEEC06F0040E326EE50EE82EFED7322E04
:100C7000FCD700F0326E300E306E3250AEEC06F023
:100C8000326E200E306E3250AEEC06F0040E326E34
:100C9000E50EE82EFED7322EFCD700F0326E0C0E99
:100CA000306E3250AEEC06F0326E140E306E3250B2
:100CB000AEEC06F0326E060E306E3250AEEC06F040
:100CC000326E010E306E3250AEEC06F01200FFFFB5
:100CD000FFFF0350F00B616E046E030E016E0450B3
:100CE00061C002F02FEC08F06184046E030E016E07
:100CF000045061C002F02FEC08F06194046E030E02
:100D0000016E045061C002F02FEC08F00338F00BC4
:100D1000F00B616E046E030E016E045061C002F0B0
:100D20002FEC08F06184046E030E016E045061C064
:100D300002F02FEC08F06194046E030E016E045073
:100D400061C002F02FEC08F0040E046EE50EE82EF0
:100D5000FED7042EFCD700F01200FFFFFFFF30503B
:100D6000F00B616E316E030E2E6E315061C02FF0AC
:100D700025EC08F06184316E030E2E6E315061C097
:100D80002FF025EC08F06194316E030E2E6E315079
:100D900061C02FF025EC08F03038F00BF00B616EDD
:100DA000316E030E2E6E315061C02FF025EC08F02D
:100DB0006184316E030E2E6E315061C02FF025EC30
:100DC00008F06194316E030E2E6E315061C02FF029
:100DD00025EC08F0040E316EE50EE82EFED7312E1C
:100DE000FCD700F01200FFFFFFFF0F0E926E010E06
:100DF000936E000E816E800E946E000E826E000E59
:100E0000956E000E836E000E966E010ED56EB00EBE
:100E1000F26E000ED76E9C0ED66E14EC06F0000E2D
:100E20005A6E000E596E000E5D6E000E5E6E53C05F
:100E300047F054C048F055C049F056C04AF02EEC77
:100E400007F04D6E000E2E6E4D504E6E000E2F6E42
:100E50004E5025EC08F0FFD7F9EF00F0FFFF000E31
:100E60004C6E000E4B6E54EC08F0060E336E100EF6
:100E7000326E9CEC07F04BEC08F047C03EF03F6A46
:100E80007BEC03F0060E336E200E326E9CEC07F006
:100E900048C03EF03F6A7BEC03F0060E336E200E36
:100EA000326E9CEC07F049C03EF03F6A7BEC03F0E9
:100EB000060E336E200E326E9CEC07F04AC03EF0F8
:100EC0003F6A7BEC03F01200FFFFFFFF000E1F6E76
:100ED000000E1E6E39EC08F0060E066E100E056E42
:100EE000CBEC07F042EC08F01AC011F0126A12ECD9
:100EF00003F0060E066E200E056ECBEC07F01BC04D
:100F000011F0126A12EC03F0060E066E200E056E4A
:100F1000CBEC07F01CC011F0126A12EC03F0060EC5
:100F2000066E200E056ECBEC07F01DC011F0126AA4
:100F300012EC03F01200FFFFFFFF000E376E000EF1
:100F4000366E00D036503224346EE86A36BEE86819
:100F50003320356E34C0F6FF35C0F7FF0800FFFFC1
:100F6000F5CF30F046EC04F0364A372A36503224BA
:100F7000346E000E3320356E34C0F6FF35C0F7FFF7
:100F80000800FFFFF5500009D8A401D001D0DAD73E
:100F900000D01200FFFFFFFF000E0A6E000E096E68
:100FA00000D009500524076EE86A09BEE8680620EB
:100FB000086E07C0F6FF08C0F7FF0800FFFFF5CF77
:100FC00003F0E4EC03F0094A0A2A09500524076EED
:100FD000000E0620086E07C0F6FF08C0F7FF0800E5
:100FE000FFFFF5500009D8A401D001D0DAD700D016
:100FF0001200FFFF00EE4FF0140EEE6AE806FDE16E
:10100000BA0EF66E100EF76E000EF86E00EE80F05F
:1010100010EE11F00900F5CFEEFFE550E150FAE1D6
:10102000CB0EF66E100EF76E000EF86E00EE63F04B
:1010300010EE11F00900F5CFEEFFE550E150FAE1B6
:10104000000EF86E0001F4EF06F0FFFF2FC083FFE3
:1010500081882EC082FF819881881200FFFFFFFFE8
:1010600002C083FF818801C082FF819881881200BD
:10107000FFFFFFFF056E800E036E055068EC06F063
:101080001200FFFFFFFF056EC00E036E055068ECF7
:1010900006F01200FFFFFFFF326EC00E306E3250BE
:1010A000AEEC06F01200FFFFFFFF326E800E306ED6
:1010B0003250AEEC06F01200FFFF49522052656D2F
:1010C0006F746520546573742020003031323334DE
:0C10D000353637383956414C55453A004A
:00000001FF
